:020000040000FA
:06000000E4EF03F0120022
:020006001200E6
:0600080031EF00F01200D0
:02000E000100EF
:0C001000E4070000C00000002E0000000B
:04001C00720ED36E1F
:10002000D3A4FED79E90CD80CD9ACD989E929D82EE
:10003000C70ECB6E040ECA6E050EBD6EF28C9D848B
:10004000F28E93869384C168F19E929092929294DC
:100050009296929C929E93800001010EEC6FFFD7C6
:100060001200DACFE4FFE2CFDAFFE9CFE4FFEACF14
:10007000E4FFF6CFE4FFF7CFE4FFF3CFE4FFF4CFE4
:10008000E4FFFACFE4FF00EE00F0100EE80403E313
:10009000EECFE4FFFBD7E6529EA2C9D29E920001AA
:1000A000ED2BED51640801E396D2010EED6FCF51B7
:1000B000000801E2CF0781B011D00001F851040B14
:1000C0000AE10001CF5107E10A0ECF6FD02BD051CA
:1000D000060801E2D06B0001F88502D00001F89516
:1000E0000001D05101E0E2D0899C899EEC056FE1CE
:1000F000EC6BD151D55DD251D65902E2EA6B0ED0EC
:10010000D5C0DDF0D6C0DEF0D1C0D5F0D2C0D6F07B
:10011000DDC0D1F0DEC0D2F0010EEA6FD551D15D65
:10012000E06FD651D259E16FD351D15D126ED251E9
:10013000D455136ED351D15D146ED251D455156E72
:10014000140E0B6E0C6A14C006F015C007F0BEEC5E
:1001500003F006C014F007C015F01450125C106EC6
:1001600015501358116E040E0F0B05E0D890113284
:100170001032E806FBE110C0E3F00001D551D35D79
:10018000126ED451D655136ED551D35D146ED45121
:10019000D655156E140E0B6E0C6A14C006F015C001
:1001A00007F0BEEC03F006C014F007C015F01450C1
:1001B000125C106E15501358116E040E0F0B05E0F3
:1001C000D89011321032E806FBE110C0E4F00001D3
:1001D000D751DB5DD851DC5902E2EB6B0ED0DBC0AE
:1001E000DDF0DCC0DEF0D7C0DBF0D8C0DCF0DDC075
:1001F000D7F0DEC0D8F0010EEB6FDB51D75DE56FB5
:10020000DC51D859E66FD951D75D126ED851DA5505
:10021000136ED951D75D146ED851DA55156E140E80
:100220000B6E0C6A14C006F015C007F0BEEC03F0AC
:1002300006C014F007C015F01450125C106E155073
:100240001358116E040E0F0B05E0D89011321032C6
:10025000E806FBE110C0E8F00001DB51D95D126E49
:10026000DA51DC55136EDB51D95D146EDA51DC5571
:10027000156E140E0B6E0C6A14C006F015C007F054
:10028000BEEC03F006C014F007C015F01450125C69
:10029000106E15501358116E040E0F0B05E0D89018
:1002A00011321032E806FBE110C0E9F00001D00580
:1002B00006E1899C898EC6C0D1F0C7C0D2F0020E7B
:1002C000D05D06E1898C898EC6C0D3F0C7C0D4F05A
:1002D000030ED05D06E1898C899EC6C0D5F0C7C0EB
:1002E000D6F0040ED05D06E1899C898EC8C0D7F097
:1002F000C9C0D8F0050ED05D06E1898C898EC8C0D2
:10030000D9F0C9C0DAF0060ED05D08E1898C899E6B
:10031000C8C0DBF0C9C0DCF0010EEC6FE26BD3515A
:10032000D15D126ED251D455136E140E0B6E0C6A41
:1003300012C006F013C007F0BEEC03F006C012F0C6
:1003400007C013F00001D3511224106ED4511320B2
:10035000116EC651105CC751115835E2E351166E4B
:10036000176AD351C65D126EC751D455136ED3515F
:10037000D15D146ED251D455156E140E0B6E0C6AED
:1003800014C006F015C007F0BEEC03F006C014F070
:1003900007C015F01450125C106E15501358116EF2
:1003A00010C006F011C007F016C00BF017C00CF01B
:1003B000BEEC03F006C0E2F00001EA510001E8B033
:1003C000F881E8A0F8910001D551D35D126ED451A7
:1003D000D655136E140E0B6E0C6A12C006F013C0C5
:1003E00007F0BEEC03F006C012F007C013F00001E6
:1003F0001250D35D106E1350D459116E1050C65D5B
:100400001150C75939E2E451166E176AC651D35DCF
:10041000126ED451C755136ED551D35D146ED4519D
:10042000D655156E140E0B6E0C6A14C006F015C06E
:1004300007F0BEEC03F006C014F007C015F014502E
:10044000125C106E15501358116E10C006F011C0DA
:1004500007F016C00BF017C00CF0BEEC03F006C09E
:10046000E2F00001EA5102E0000E01D0010E0001AD
:10047000E8B0F881E8A0F8910001E76BD951D75DA9
:10048000126ED851DA55136E140E0B6E0C6A12C030
:1004900006F013C007F0BEEC03F006C012F007C070
:1004A00013F00001D9511224106EDA511320116E8D
:1004B000C851105CC951115835E2E851166E176ADF
:1004C000D951C85D126EC951DA55136ED951D75D35
:1004D000146ED851DA55156E140E0B6E0C6A14C0DA
:1004E00006F015C007F0BEEC03F006C014F007C01C
:1004F00015F01450125C106E15501358116E10C088
:1005000006F011C007F016C00BF017C00CF0BEECDF
:1005100003F006C0E7F00001EB510001E8B0F883FA
:10052000E8A0F8930001DB51D95D126EDA51DC5579
:10053000136E140E0B6E0C6A12C006F013C007F097
:10054000BEEC03F006C012F007C013F00001125019
:10055000D95D106E1350DA59116E1050C85D1150EC
:10056000C95939E2E951166E176AC851D95D126E40
:10057000DA51C955136EDB51D95D146EDA51DC5571
:10058000156E140E0B6E0C6A14C006F015C007F041
:10059000BEEC03F006C014F007C015F01450125C56
:1005A000106E15501358116E10C006F011C007F0F0
:1005B00016C00BF017C00CF0BEEC03F006C0E7F05D
:1005C0000001EB5102E0000E01D0010E0001E8B085
:1005D000F883E8A0F8930001DF2BDF51100802E256
:1005E000010EDF6FDF51E25D0DE3140EE25D0AE202
:1005F0000001F8B102D089808992F8A102D08990D7
:10060000898202D0899089920001DF51E75D0DE374
:10061000140EE75D0AE20001F8B302D089848996DE
:10062000F8A302D08994898602D0899489969EA4E1
:100630003CD09E940001CE0517E1040EBD6ECE6B3A
:10064000C251BE5CCC6FC351BF58CD6FBECFC0F09E
:10065000BFCFC1F0100ECC5D270ECD5904E2CCC047
:10066000C8F0CDC0C9F021D0050EBD6E010ECE6F11
:10067000C051BE5CC46FC151BF58C56FBECFC2F080
:10068000BFCFC3F0100ED880CC55270ECD5504E255
:10069000C4C0C6F0C5C0C7F0100ECC5D270ECD5942
:1006A00004E2C4C0CAF0C5C0CBF0E55200EE0FF0C2
:1006B000100EE80403E3E5CFEDFFFBD7E5CFFAFF2B
:1006C000E5CFF4FFE5CFF3FFE5CFF7FFE5CFF6FF8A
:0E06D000E5CFEAFFE5CFE9FFE5CFDAFF110045
:0206DE000E0EFE
:1006E000F66E000EF76E000EF86E00010900F55070
:1006F000F36F0900F550F46F03E1F36701D03DD0CB
:100700000900F550EE6F0900F550EF6F0900F55044
:10071000F06F09000900F550E96E0900F550EA6E26
:10072000090009000900F550F16F0900F550F26F5A
:1007300009000900F6CFF5F0F7CFF6F0F8CFF7F0A3
:10074000EEC0F6FFEFC0F7FFF0C0F8FF0001F15375
:1007500002E1F25307E00900F550EE6EF107F8E20E
:10076000F207F9D7F5C0F6FFF6C0F7FFF7C0F8FFBC
:0C0770000001F307000EF45BBFD712007D
:04077C00036A026AA0
:10078000100EE76ED89006360736023603360B5049
:10079000025C0C50035805E30B50025E0C50035AE8
:0807A000062AE72EF0D7120033
:0807A800000EF36E00EE00F0FC
:1007B000010E01D81200EA6002D0EE6AFCD7F350B5
:0807C000E9601200EE6AFCD7AB
:0807C80010EE80F020EE80F03D
:1007D000F86A0F9C6FEC03F003EC00F00EEC00F0F5
:0407E000FBD7120031
:0C07E40000000000000000000000000009
:1007F00000000100004D09EB0CBE10E607820B8FD4
:100800000F000000D007000A0AD007000A0A010101
:020810000100E5
:020000040030CA
:01000100C836
:010003001EDE
:010006008178
:00000001FF
